:100000009F01831691010730831299003A308316BD
:100010008500333087008716071683129601161362
:10002000961616159701971717131716971591011E
:10003000911503309300013092006F10EF10C4222D
:10004000A60080302605031D82292608E3226130A0
:100050002602031C33287A302602031903100318E2
:100060003328E030A607BF302607031D45285E224F
:10007000A7005E22A9004122EF1E44282708C822BB
:10008000DB222908C822DE227F29BE302607031D75
:1000900052285E22AE004122EF1E51282E08C822AF
:1000A000DE227F29BD302607031D5A284122EF1A80
:1000B000DE227F29BC302607031D73284122EF1E54
:1000C0007228DE22FF30E021FE21AE006F1D6B287A
:1000D0004030E3227128EF1D6F283130E3222E08D3
:1000E000C822DE227F29BA302607031D8A28412232
:1000F000EF1E89286F116F198828FE21AE00DB22C0
:100100006F1D85284030E32287282E08C8227B28CF
:10011000DE227F29B7302607031D92284122EF1ADD
:10012000AF217F29B6302607031DA0286122412276
:10013000EF1E9F282308C8222408C822DE227F2918
:10014000B0302607031DE3285E22AA004122EF1EDD
:10015000E228AC01A80110302C020318E2282A087A
:10016000C8222808C8223A30E3220030E021FE21CC
:100170002A08E021FE212808E021FE21FE2101308D
:10018000E021FE210830E021FE210830B900FE21E7
:10019000AE00DB226F1DCF284030E322D1282E088D
:1001A000C822FE21AE006F1DD8284030E322DA2895
:1001B0002E08C822B90BC728FE21DE22AC0A08305F
:1001C000A807AB287F29AE302607031DF12861223E
:1001D0004122EF1EF0282308C8222408C822DE226C
:1001E0007F29AD302607031D1A295E22A90041226E
:1001F000EF1E1929DE222908EF21FE21AE006F1D16
:1002000004294030E32206292E08C822FE21AE0030
:100210006F1D0D294030E3220F292E08C822FE2130
:10022000AE006F1D16294030E32218292E08C8227F
:10023000DE227F29A9302607031D2C2961225E2298
:10024000AE004122EF1E2B292308C8222408C82211
:100250002E08C822DE227F29A8302607031D542934
:100260005E22AE004122EF1E53292E08E021FE211E
:10027000AE006F1D3E294030E32240292E08C822DF
:10028000FE21AE006F1D47294030E32249292E0888
:10029000C822FE21AE006F1D50294030E3225229B2
:1002A0002E08C822DE227F29A6302607031D7029CA
:1002B0004122EF1E6F290130A900290803196F2977
:1002C0002908EF21FE21AE00FE21AE006F196D2935
:1002D0002908C8223A30E322AF21A90A5D297F29E3
:1002E000C6302607031D78294122EF1ADE227F2916
:1002F000F330260703197F293F30E322DE223E3008
:10030000E322AE29260CB900B90C390C0739AD002F
:1003100007302605AB006F12261B6F162D08031938
:10032000A0292D08B900C422A6006F1E9B296F12B8
:100330002608EF219D292608E021FE21B90B9329EB
:100340002B080319AE292B08B900FE21A6006F194E
:10035000FC306F1D2608E322B90BA5291D28FE30AD
:10036000DA21AF000530BA00FD30DA21AF002F08E6
:10037000C822DB22BA0BB42902302F05031DC62187
:1003800001302F05031DC621DE220034DB22FD30A3
:10039000DA21B0003008C8223A30E3222230E322CA
:1003A0003008BB00FD30DA21E322BB0BD22922301A
:1003B000E3220034B1003108E021FE21FE210800D3
:1003C000B2000430BC00033032051822B20CB20C6B
:1003D0003F30B205BC0BE329043018220034B300CF
:1003E0000430BD00033033051822B30CB30C3F308A
:1003F000B305BD0BF2290530182200346F110F3000
:10040000BE001430BF0006301822A518122AEF11C2
:100410002518EF150430C00000301822C00B0C2A3C
:1004200025080800BF0B032ABE0B012A6F150034F4
:10043000B40005108711071134190514B418871575
:1004400034180715051D282A05118518252A2B2A79
:100450000515851C292AA50DA50DFC30A5058718B5
:10046000A514071825140034C422B5003508E3226A
:10047000F3303507031D3F2AEF140A30E322350815
:1004800008006F1C452AEF120800EF185C2A34227E
:10049000B600F330360703195B2AF7303607031925
:1004A0005B2AE030360703195B2A6F142130E32200
:1004B000DE22EF120800452AEF1608006122240808
:1004C0000800A301A4012030B700EF18B62AE030DD
:1004D000370703196F2AF7303707031D722A3422B2
:1004E000B700672A30303702031C7C2A39303702C4
:1004F00003190310031CA42A41303702031C862A67
:100500004630370203190310031CA02A613037025A
:10051000031C902A6630370203190310031C9C2A1F
:10052000E030370703199A2AF730370703199A2A58
:10053000EF1C6F1400349F2AA9303707B800A32A94
:10054000C9303707B800A72AD0303707B800230EC4
:10055000C100F030C105240E0F394104A300240E60
:10056000F0393804A4003422B700722A0034FF3076
:10057000C300FF30C4008C1EBF2A14080800C40B3F
:10058000BB2AC30BB92AFC348C1EC42A14080800E9
:10059000A000200E0F39D0220F302005D0220034C9
:1005A000A1000A30210203183730031C3030A107A4
:1005B0002108E32200342030E32200340D30E3220E
:1005C0000A30E3220034A2008C1CE42A22089500A1
:0205D0000034F5
:02400E00D230AE
:00000001FF
